:020000040000FA
:040000000DEF00F010
:04000800A4EF08F069
:0800180010000F01D0B014EF3D
:1000200000F0D080000133840F01D0B61BEF00F048
:10003000D086000133820F01D39ED38CD38AD3980C
:10004000D396D382D3900F019B9E9B8C0001806A34
:10005000896A816A8A6A826A8B6A0F01936A938AC3
:10006000939C938E8A6A8A8A8A9C8A8E000EB06ECE
:100070000F01CF0EAF6E0F01B8860F01AC84AC98A4
:100080000F010F01AC8A0F01AB88000178EC06F07C
:100090000F01BA8EBA8ABA880F01BB6A0F01BC6A17
:1000A0000F01200EC16E0F01CA0E946E0F017E80EB
:1000B0007E827E847E867E987E8A7E9C7E8E0F01E6
:1000C0007F807F827F947F960F01D58ED58CD58AD5
:1000D000D588D586D59AD5860F019D6A9D800F015A
:1000E000A0980F018188818C818E0F01829082847B
:1000F00082881F6A206A1E6A216A000194EC05F05A
:1001000033980001026A3390029253A00282276A58
:100110000F01CD9ECD8ACD88CD96CD94CD92CD8048
:10012000000E0F01CF6E0F01CE6E0F019E900001E9
:100130000F01F26AF28CF28E0F01D18053A298EC7B
:1001400008F00001040033A2C1EF00F0570E25ECC7
:1001500004F0610E25EC04F0740E25EC04F0630E3F
:1001600025EC04F0680E25EC04F0640E25EC04F098
:100170006F0E25EC04F0670E25EC04F086EC04F01D
:100180003392E1EF00F033A4E1EF00F0420E25ECF2
:1001900004F0720E25EC04F06F0E25EC04F0770EDF
:1001A00025EC04F06E0E25EC04F06F0E25EC04F047
:1001B000750E25EC04F0740E25EC04F086EC04F0CA
:1001C0003394FF0E155CD8B419EF01F002A019EFBB
:1001D00001F0029078EC0CF0020E1D6EF9EC03F0C9
:1001E000000123EC06F000013FEC06F00001000ED8
:1001F000426E1550416E010E406E110E3F6EA1EC25
:1002000006F04250086E4150036E2C50426E2D5045
:10021000416E0850406E03503F6E9CEC06F00001AA
:1002200042AE17EF01F08290338619EF01F0828021
:10023000339600010F0E245CD8A485EF01F0000175
:10024000540E25EC04F0690E25EC04F06D0E25EC3F
:1002500004F0650E25EC04F0720E25EC04F0200E7F
:1002600025EC04F0310E25EC04F0200E25EC04F012
:10027000355030EC04F03A0E25EC04F0365030ECFA
:1002800004F0200E25EC04F0375030EC04F0B00EF2
:1002900025EC04F0430E25EC04F0200E25EC04F0D0
:1002A000200E25EC04F0540E25EC04F0690E25EC2C
:1002B00004F06D0E25EC04F0650E25EC04F0720ED2
:1002C00025EC04F0200E25EC04F0320E25EC04F0B1
:1002D000200E25EC04F0385030EC04F03A0E25ECFA
:1002E00004F0395030EC04F0200E25EC04F03A50C4
:1002F00030EC04F0B00E25EC04F0430E25EC04F0D5
:1003000086EC04F00001F5EF03F00D0E245CD8A498
:1003100009EF02F00001540E25EC04F0690E25EC03
:1003200004F06D0E25EC04F0650E25EC04F0720E61
:1003300025EC04F0200E25EC04F0310E25EC04F041
:10034000200E25EC04F0480E25EC04F06F0E25EC91
:1003500004F0750E25EC04F0720E25EC04F03F0E4F
:1003600025EC04F086EC04F08CEC06F03B50356E86
:1003700086EC04F04D0E25EC04F0690E25EC04F03B
:100380006E0E25EC04F0750E25EC04F0740E25ECD1
:1003900004F0650E25EC04F03F0E25EC04F086EC2D
:1003A00004F08CEC06F03B50366E86EC04F0540EF4
:1003B00025EC04F0650E25EC04F06D0E25EC04F040
:1003C000700E25EC04F0650E25EC04F0720E25ECA1
:1003D00004F0610E25EC04F0740E25EC04F0750EAB
:1003E00025EC04F0720E25EC04F0650E25EC04F00B
:1003F0003F0E25EC04F086EC04F08CEC06F03B504C
:10040000376E86EC04F0000154EC05F00001F5EFC6
:1004100003F00E0E245CD8A48DEF02F00001540E00
:1004200025EC04F0690E25EC04F06D0E25EC04F0CB
:10043000650E25EC04F0720E25EC04F0200E25EC80
:1004400004F0320E25EC04F0200E25EC04F0480EEA
:1004500025EC04F06F0E25EC04F0750E25EC04F08D
:10046000720E25EC04F03F0E25EC04F086EC04F04F
:100470008CEC06F03B50386E86EC04F04D0E25EC0B
:1004800004F0690E25EC04F06E0E25EC04F0750EF8
:1004900025EC04F0740E25EC04F0650E25EC04F058
:1004A0003F0E25EC04F086EC04F08CEC06F03B509B
:1004B000396E86EC04F0540E25EC04F0650E25EC44
:1004C00004F06D0E25EC04F0700E25EC04F0650EC2
:1004D00025EC04F0720E25EC04F0610E25EC04F01E
:1004E000740E25EC04F0750E25EC04F0720E25EC6C
:1004F00004F0650E25EC04F03F0E25EC04F086ECCC
:1005000004F08CEC06F03B503A6E86EC04F00001EF
:1005100054EC05F00001F5EF03F03550215CD8A450
:1005200099EF02F036501E5CD8A499EF02F03750D4
:10053000156E3850215CD8A4A5EF02F039501E5C2E
:10054000D8A4A5EF02F03A50156E110E245CD8A481
:10055000F3EF02F0010E1D6EF9EC03F00001200E26
:1005600025EC04F01AEC06F0020E1D6EF9EC03F017
:100570000001200E25EC04F01AEC06F0030E1D6EAF
:10058000F9EC03F00001200E25EC04F01AEC06F063
:10059000050E1D6EF9EC03F00001200E25EC04F0B1
:1005A0001AEC06F0070E1D6EF9EC03F00001200EA8
:1005B00025EC04F01AEC06F0080E1D6EF9EC03F0C1
:1005C0000001200E25EC04F01AEC06F0090E1D6E59
:1005D000F9EC03F00001200E25EC04F01AEC06F013
:1005E000000186EC04F0100E245CD8A400EF03F0A8
:1005F0001C5030EC04F086EC04F00001F5EF03F041
:10060000080E245CD8A40CEF03F06EEC06F0000199
:1006100086EC04F0F5EF03F00001020E245CD8A490
:1006200017EF03F01C500F01BE6EF5EF03F0000151
:10063000010E245CD8A427EF03F0F9EC03F00001CD
:100640001AEC06F0000186EC04F0F5EF03F000016F
:10065000030E245CD8A43BEF03F0F9EC03F0000197
:1006600023EC06F00001F5EC05F0000186EC04F047
:100670000001F5EF03F000010A0E245CD8A452EF4C
:1006800003F0F9EC03F0000123EC06F000013FEC6D
:1006900006F0000104EC06F0000186EC04F0000115
:1006A000F5EF03F000010C0E245CD8A467EF03F013
:1006B000155030EC04F00001B00E25EC04F0430EB0
:1006C00025EC04F086EC04F00001F5EF03F00001E6
:1006D000040E245CD8A495EF03F01650000AD8A4A9
:1006E00075EF03F08188F5EF03F01650010AD8A4E6
:1006F0007DEF03F0818CF5EF03F01650020AD8A4C9
:1007000085EF03F08280F5EF03F01650030AD8A4BA
:100710008DEF03F08284F5EF03F01650040AD8A49D
:10072000F5EF03F08288F5EF03F00001050E245C7D
:10073000D8A4C3EF03F01650000AD8A4A3EF03F027
:100740008198F5EF03F01650010AD8A4ABEF03F03F
:10075000819CF5EF03F01650020AD8A4B3EF03F022
:100760008290F5EF03F01650030AD8A4BBEF03F014
:100770008294F5EF03F01650040AD8A4F5EF03F0C5
:100780008298F5EF03F00001090E245CD8A4E8EF8D
:1007900003F01650000AD8A4D5EF03F08050080BE0
:1007A000D8A4E1EF03F0DEEF03F0010AD8A4F5EFDF
:1007B00003F08050200BD8A4E1EF03F0300EE2EFFD
:1007C00003F0310E25EC04F086EC04F0F5EF03F0B5
:1007D0000001070E245CD8A4A1EF00F0145030EC07
:1007E00004F086EC04F0F5EF03F00001246AA1EFB9
:1007F00000F000011D500F0B1A6E1A461A461A50CF
:100800000F01C26AC26EC2800F01C186C194C1923B
:10081000C1900F01C08EC09AC098C086C094C0928B
:10082000C0900001FF0E006E002E14EF04F0C28293
:10083000C2B218EF04F00F01C4500001256E0F0181
:10084000C3500001266E1200300F000102A21200F8
:100850000F01AD6E0F01ACA22BEF04F000011200EE
:100860000284036E046A640E035ED8A03BEF04F0BA
:10087000042A33EF04F0000E045CD8B444EF04F013
:100880000294045024EC04F0640E0326046A0A0E59
:10089000035ED8A04FEF04F0042A47EF04F0000EE7
:1008A000045CD8A457EF04F002B45AEF04F00450EB
:1008B00024EC04F00A0E0326035024EC04F012008A
:1008C000000145EC08F002840E507CEC04F00F505F
:1008D0007CEC04F010507CEC04F011507CEC04F043
:1008E00002AC77EF04F02E0E25EC04F0029C02948B
:1008F00012507CEC04F0120002A482EF04F00F0B03
:10090000D8B4120024EC04F0029412000D0E25EC71
:1009100004F00A0E25EC04F0120000013D50A96E0F
:10092000000EAA6E3E50A86EA69EA69CA684F29EBD
:10093000550EA76EAA0EA76EA682F28E0F01A6B262
:100940009EEF04F0A694A6EC04F0120048EC05F02B
:1009500000013E500F01A85CD8A4B1EF04F00001E3
:100960001200B5EC04F0000112000001650E25EC48
:1009700004F0650E25EC04F0700E25EC04F0720E08
:1009800025EC04F06F0E25EC04F06D0E25EC04F060
:10099000200E25EC04F0770E25EC04F0720E25EC09
:1009A00004F0690E25EC04F0740E25EC04F0650EDD
:1009B00025EC04F0200E25EC04F0720E25EC04F07A
:1009C000650E25EC04F0730E25EC04F0750E25EC95
:1009D00004F06C0E25EC04F0740E25EC04F0200EEF
:1009E00025EC04F0610E25EC04F0640E25EC04F017
:1009F000640E25EC04F0720E25EC04F0650E25EC77
:100A000004F0730E25EC04F0730E25EC04F03D0E9B
:100A100025EC04F03D5030EC04F0200E25EC04F001
:100A20006F0E25EC04F0720E25EC04F0690E25EC37
:100A300004F0670E25EC04F0690E25EC04F06E0E50
:100A400025EC04F0610E25EC04F06C0E25EC04F0AE
:100A50003D0E25EC04F03E5030EC04F0200E25EC69
:100A600004F0720E25EC04F0650E25EC04F0610E26
:100A700025EC04F0640E25EC04F03D0E25EC04F0AA
:100A800048EC05F0000130EC04F086EC04F01200B4
:100A900000013D500F01A96E0F01A69EA69CA680E5
:100AA0000F01A850A85012000001000E3D6E145016
:100AB0003E6E8DEC04F000013D2A1C503E6E8DEC24
:100AC00004F000013D2A15503E6E8DEC04F000014B
:100AD0003D2A35503E6E8DEC04F000013D2A365023
:100AE0003E6E8DEC04F000013D2A37503E6E8DECD9
:100AF00004F000013D2A38503E6E8DEC04F00001F8
:100B00003D2A39503E6E8DEC04F000013D2A3A50EA
:100B10003E6E8DEC04F000010C0E3D6E53503E6EA7
:100B20008DEC04F0000112000001FF0E3D6E48EC58
:100B300005F000017B0AD8B4B0EF05F00001AF0E5C
:100B4000146E320E1C6E000E506E516E526E536E4D
:100B50007B0E3E6EFF0E3D6E8DEC04F00001120028
:100B60000001000E3D6E48EC05F00001146E3D2AB8
:100B700048EC05F000011C6E3D2A48EC05F0000130
:100B8000156E3D2A48EC05F00001356E3D2A48EC13
:100B900005F00001366E3D2A48EC05F00001376E85
:100BA0003D2A48EC05F00001386E3D2A48EC05F07E
:100BB0000001396E3D2A48EC05F000013A6E3D2AED
:100BC00048EC05F00001506E3D2A48EC05F00001AC
:100BD000516E3D2A48EC05F00001526E3D2A48EC6A
:100BE00005F00001536E0001120000012A500C6E46
:100BF0002B500D6E60EC04F000016D0E25EC04F03E
:100C0000560E25EC04F01200000102A60BEF06F0D0
:100C10002D0E25EC04F000012E500C6E2F500D6EA1
:100C200060EC04F00001B00E25EC04F0430E25EC5E
:100C300004F01200000125500C6E26500D6E60EC81
:100C400004F0000112000F0E406EF00E3F6E2550B2
:100C5000426E2650416E36EC08F04150426E4450D0
:100C6000416E000E406E040E3F6EB1EC06F00001C6
:100C70004250096E2A6E41500A6E2B6E12002A50A5
:100C8000426E2B50416E000E406E0A0E3F6EB1EC6C
:100C900006F0000142502C6E41502D6E010E406E48
:100CA000110E3F6E9CEC06F0000142502E6E41503A
:100CB0002F6E0296000142AE120002862C50406E4A
:100CC0002D503F6E010E426E110E416E9CEC06F0EF
:100CD000000142502E6E41502F6E1200215030EC18
:100CE00004F03A0E25EC04F01E5030EC04F0120033
:100CF0000F01CC6A0F01650ECB6E0001320E1C6E27
:100D00000F01BE6E0C0E0F01BD6E0F01CA6ACA90B4
:100D1000CA92CA8400011200000133800F0E176EC0
:100D2000040033B090EF06F03B5012003F1E3F2A04
:100D3000D8B44006401E000C3F1E3F2AD8B44006DF
:100D4000401E3F504126D8B0422A40504226000C57
:100D5000100E086E4250466E4150456E426A416A1E
:100D6000000CA8EC06F0446A436AD8904536463633
:100D7000433644364050445CD8A4C1EF06F03F509F
:100D8000435CD8A0CBEF06F03F50435ED8A04406AA
:100D90004050445ED88041364236D890453646367B
:100DA000433644364050445CD8A4D9EF06F03F5057
:100DB000435CD8A0E3EF06F03F50435ED8A0440662
:100DC0004050445ED88041364236D890453646364B
:100DD000433644364050445CD8A4F1EF06F03F500F
:100DE000435CD8A0FBEF06F03F50435ED8A044061A
:100DF0004050445ED88041364236D890453646361B
:100E0000433644364050445CD8A409EF07F03F50C5
:100E1000435CD8A013EF07F03F50435ED8A04406D0
:100E20004050445ED88041364236D89045364636EA
:100E3000433644364050445CD8A421EF07F03F507D
:100E4000435CD8A02BEF07F03F50435ED8A0440688
:100E50004050445ED88041364236D89045364636BA
:100E6000433644364050445CD8A439EF07F03F5035
:100E7000435CD8A043EF07F03F50435ED8A0440640
:100E80004050445ED88041364236D890453646368A
:100E9000433644364050445CD8A451EF07F03F50ED
:100EA000435CD8A05BEF07F03F50435ED8A04406F8
:100EB0004050445ED88041364236D890453646365A
:100EC000433644364050445CD8A469EF07F03F50A5
:100ED000435CD8A073EF07F03F50435ED8A04406B0
:100EE0004050445ED88041364236D890453646362A
:100EF000433644364050445CD8A481EF07F03F505D
:100F0000435CD8A08BEF07F03F50435ED8A0440667
:100F10004050445ED88041364236D89045364636F9
:100F2000433644364050445CD8A499EF07F03F5014
:100F3000435CD8A0A3EF07F03F50435ED8A044061F
:100F40004050445ED88041364236D89045364636C9
:100F5000433644364050445CD8A4B1EF07F03F50CC
:100F6000435CD8A0BBEF07F03F50435ED8A04406D7
:100F70004050445ED88041364236D8904536463699
:100F8000433644364050445CD8A4C9EF07F03F5084
:100F9000435CD8A0D3EF07F03F50435ED8A044068F
:100FA0004050445ED88041364236D8904536463669
:100FB000433644364050445CD8A4E1EF07F03F503C
:100FC000435CD8A0EBEF07F03F50435ED8A0440647
:100FD0004050445ED88041364236D8904536463639
:100FE000433644364050445CD8A4F9EF07F03F50F4
:100FF000435CD8A003EF08F03F50435ED8A04406FE
:101000004050445ED88041364236D8904536463608
:10101000433644364050445CD8A411EF08F03F50AA
:10102000435CD8A01BEF08F03F50435ED8A04406B5
:101030004050445ED88041364236D89045364636D8
:10104000433644364050445CD8A429EF08F03F5062
:10105000435CD8A033EF08F03F50435ED8A044066D
:101060004050445ED88041364236000CA8EC06F071
:1010700046324532D8B0A1EC06F042324132443219
:101080004332082E38EF08F0000C0C504B6E0D5018
:101090004C6E4B30E8323F0B4E6E180D030E4B1664
:1010A000F3504C26F4504B22E80E4C5E030E4B5A84
:1010B00008E34E2AE80E4C5E030E4B5A02E34E2A1A
:1010C00004D0E80E4C26030E4B224C344B34070B55
:1010D0004F6E1C0D4C9EF3504C2605E3380E4C26EB
:1010E0004F2A4F2A08D0640E4C5E04E34F2A4C5E10
:1010F00001E34F4A4C264E50CD0D200EF402F45021
:101100004D6E0A0DF3504E5E4C50CD0D200EF40284
:10111000F4504B6E0A0DF3504C5E4D500E6E4E5017
:101120000F6E4F50106E4B50116E4C50126E1200DD
:1011300033B812000F01AB8E0F01AC8A0F019D8AEC
:10114000338811EC0DF01200496ED838D86A4A6E17
:10115000FA50476E000104009EA0D6EF08F0029EF0
:101160001F2ED0EF08F0028E050E1F6E202A3C0EB7
:10117000205CD8A4D0EF08F0000198EC08F0000142
:10118000206A1E2A02803C0E1E5CD8A4D0EF08F014
:101190001E6A212A180E215CD8A4D0EF08F0216A1B
:1011A0003C0ECF6E1450CE6ECD8ACD880F01ABA40D
:1011B000DCEF08F0DFEF08F0ABA2E8EF08F0AB944B
:1011C000AB92AB98AB88070E25EC04F05EEF0CF009
:1011D0009EAA5EEF0CF033A0F0EF08F099EF09F053
:1011E000570EAE5CD8B42BEF0AF0550EAE5CD8B4F7
:1011F00032EF0AF05F0EAE5CD8B439EF0AF0500E51
:10120000AE5CD8B440EF0AF0490EAE5CD8B447EFFC
:101210000AF0430EAE5CD8B44EEF0AF0276A02A281
:101220005EEF0CF0610EAE5CD8B4D9EF0BF0420E5D
:10123000AE5CD8B489EF0AF0620EAE5CD8B4C0EFF1
:101240000AF0440EAE5CD8B47AEF0AF0640EAE5CDD
:10125000D8B480EF0AF0630EAE5CD8B4F5EF0BF0B3
:10126000450EAE5CD8B4FAEF0AF0650EAE5CD8B4A9
:1012700064EF0BF0670EAE5CD8B462EF0AF0470E75
:10128000AE5CD8B4EDEF0BF0480EAE5CD8B4E9EF2D
:101290000BF0680EAE5CD8B415EF0AF04C0EAE5CE5
:1012A000D8B45EEF0AF0690EAE5CD8B4F9EF0BF07B
:1012B0004D0EAE5CD8B4E5EF0BF0510EAE5CD8B479
:1012C000D5EF0BF0710EAE5CD8B425EF0AF0720EBC
:1012D000AE5CD8B4E1EF0BF0730EAE5CD8B4F1EFB6
:1012E0000BF0740EAE5CD8B468EF0AF0760EAE5C0C
:1012F000D8B4DDEF0BF0770EAE5CD8B485EF0AF012
:10130000580EAE5CD8B4D1EF0BF0780EAE5CD8B40A
:101310001FEF0AF0590EAE5CD8B46EEF0AF0790EEA
:10132000AE5CD8B419EF0AF05A0EAE5CD8B474EFC4
:101330000AF00D0EAE5CD8B4D2EF09F0300EAE5C00
:10134000D8B444EF0CF0310EAE5CD8B444EF0CF0DE
:10135000320EAE5CD8B444EF0CF0330EAE5CD8B4B1
:1013600044EF0CF0340EAE5CD8B444EF0CF0350E04
:10137000AE5CD8B444EF0CF0360EAE5CD8B444EF9B
:101380000CF0370EAE5CD8B444EF0CF0380EAE5C07
:10139000D8B444EF0CF0390EAE5CD8B444EF0CF086
:1013A0005EEF0CF0000E195CD8B45EEF0CF0010E8D
:1013B000175CD8B412EF0CF0030E175CD8B40AEF28
:1013C0000CF0040E175CD8B418EF0CF00C0E175C80
:1013D000D8B41EEF0CF0070E175CD8B424EF0CF055
:1013E000080E175CD8B428EF0CF00B0E175CD8B4BD
:1013F0003EEF0CF0050E175CD8B432EF0CF0060E81
:10140000175CD8B438EF0CF0090E175CD8B42CEF89
:101410000CF00D0E175CD8B402EF0CF00F0E175C39
:10142000D8B4FDEF0BF05EEF0CF01AEC0DF05CEFB2
:101430000CF0120E176E0F0E246E5CEF0CF00E0EF9
:10144000176E0C0E246E5CEF0CF0130E176E100E60
:10145000246E5CEF0CF0000E275CD8B45BEF0AF052
:1014600058EF0AF0010E275CD8B45BEF0AF058EF92
:101470000AF0020E275CD8B45BEF0AF058EF0AF0CE
:10148000030E275CD8B45BEF0AF058EF0AF0040EA5
:10149000275CD8B45BEF0AF058EF0AF0050E275C22
:1014A000D8B455EF0AF058EF0AF0028211EC0DF0B3
:1014B000276A5CEF0CF0272A5CEF0CF0276A029297
:1014C0005CEF0CF00A0E176E070E246E5CEF0CF04A
:1014D000020E176E080E246E5CEF0CF0100E176EE5
:1014E0000D0E246E5CEF0CF0110E176E0E0E246EB6
:1014F0005CEF0CF0140E176E110E246E5CEF0CF006
:10150000140E176E246A5CEF0CF09FEC0CF05CEF8D
:101510000CF0538054EC05F0500E25EC04F0610EF5
:1015200025EC04F0730E25EC04F0730E25EC04F0AA
:10153000770E25EC04F06F0E25EC04F0720E25EC0E
:1015400004F0640E25EC04F0200E25EC04F0650E8A
:1015500025EC04F06E0E25EC04F0610E25EC04F091
:10156000620E25EC04F06C0E25EC04F0650E25EC03
:1015700004F0640E25EC04F086EC04F05CEF0CF053
:10158000539054EC05F0500E25EC04F0610E25EC60
:1015900004F0730E25EC04F0730E25EC04F0770EC6
:1015A00025EC04F06F0E25EC04F0720E25EC04F02F
:1015B000640E25EC04F0200E25EC04F0640E25ECFE
:1015C00004F0690E25EC04F0730E25EC04F0610EB6
:1015D00025EC04F0620E25EC04F06C0E25EC04F012
:1015E000650E25EC04F0640E25EC04F086EC04F0A6
:1015F0005CEF0CF0538254EC05F0530E25EC04F034
:10160000650E25EC04F0720E25EC04F0690E25EC55
:1016100004F0610E25EC04F06C0E25EC04F0200EB5
:1016200025EC04F0700E25EC04F06F0E25EC04F0B0
:10163000720E25EC04F0740E25EC04F0200E25EC5F
:1016400004F0730E25EC04F0740E25EC04F0610E2A
:1016500025EC04F0720E25EC04F0740E25EC04F079
:10166000750E25EC04F0700E25EC04F0200E25EC30
:1016700004F0640E25EC04F0650E25EC04F06C0E0D
:1016800025EC04F0610E25EC04F0790E25EC04F055
:10169000200E25EC04F0650E25EC04F06E0E25EC12
:1016A00004F0610E25EC04F0620E25EC04F06C0EE3
:1016B00025EC04F0650E25EC04F0640E25EC04F036
:1016C00086EC04F05CEF0CF0539254EC05F0530EF2
:1016D00025EC04F0650E25EC04F0720E25EC04F008
:1016E000690E25EC04F0610E25EC04F06C0E25EC7F
:1016F00004F0200E25EC04F0700E25EC04F06F0EC3
:1017000025EC04F0720E25EC04F0740E25EC04F0C8
:10171000200E25EC04F0730E25EC04F0740E25EC7D
:1017200004F0610E25EC04F0720E25EC04F0740E4A
:1017300025EC04F0750E25EC04F0700E25EC04F099
:10174000200E25EC04F0640E25EC04F0650E25EC6B
:1017500004F06C0E25EC04F0610E25EC04F0790E1B
:1017600025EC04F0200E25EC04F0640E25EC04F0CA
:10177000690E25EC04F0730E25EC04F0610E25ECE7
:1017800004F0620E25EC04F06C0E25EC04F0650EFE
:1017900025EC04F0640E25EC04F086EC04F05CEF1C
:1017A0000CF00D0E176E57EF0CF0030E176E57EF7F
:1017B0000CF0010E176E57EF0CF0040E176E57EF7A
:1017C0000CF00C0E176E57EF0CF0070E176E57EF5C
:1017D0000CF0080E176E57EF0CF0090E176E57EF4E
:1017E0000CF0050E176E57EF0CF0060E176E57EF44
:1017F0000CF00B0E176E57EF0CF01B503B6E339036
:1018000056EF0CF01B50156E0B0E246E54EC05F0C9
:1018100056EF0CF01B501C6E020E246E54EC05F0BB
:1018200056EF0CF01B501D6E010E246E56EF0CF09F
:101830001B501D6E030E246E56EF0CF01B501D6ED8
:101840000A0E246E56EF0CF01B501E6E56EF0CF075
:101850001B50216E56EF0CF01B50146E54EC05F02B
:1018600056EF0CF01B50166E040E246E56EF0CF063
:101870001B50166E050E246E56EF0CF01B50166EA4
:10188000090E246E56EF0CF0300EAE5C186E1B5035
:101890001B261B261B261B261B261B261B261B2640
:1018A0001B2618501B26192A5EEF0CF000010001C0
:1018B0001B6A196A5EEF0CF00001176A0001F29EC4
:1018C000F29AF298F296F294F292F2909E9C9E9A7C
:1018D0009E989E969E949E929E90A19EA19AA19C57
:1018E000A1984750FA6E4A38D86E493A49381000E4
:1018F00033A61200502A3C0E505CD8A489EF0CF09D
:10190000506A512A180E515CD8A489EF0CF0516A24
:10191000522A0001090E3D6E50503E6E8DEC04F0CF
:1019200000010A0E3D6E51503E6E8DEC04F0000138
:101930000B0E3D6E52503E6E8DEC04F01200480EC0
:1019400025EC04F0650E25EC04F0610E25EC04F0A6
:10195000740E25EC04F0650E25EC04F0720E25ECF7
:1019600004F0200E25EC04F06F0E25EC04F06E0E52
:1019700025EC04F0200E25EC04F0200E25EC04F0FC
:10198000525030EC04F0200E25EC04F0640E25ECEF
:1019900004F0610E25EC04F0790E25EC04F0730ED2
:1019A00025EC04F0200E25EC04F0200E25EC04F0CC
:1019B000515030EC04F0200E25EC04F0680E25ECBC
:1019C00004F06F0E25EC04F0750E25EC04F0720E99
:1019D00025EC04F0730E25EC04F0200E25EC04F049
:1019E000200E25EC04F0505030EC04F0200E25ECD5
:1019F00004F06D0E25EC04F0690E25EC04F06E0E7B
:101A000025EC04F0750E25EC04F0740E25EC04F0C2
:101A1000650E25EC04F0730E25EC04F086EC04F062
:101A200012000001000E056E230E066E280E076ED2
:101A300023EF0DF00001000E056E1A0E066E680E03
:101A4000076E23EF0DF000010550F86E0650F76E9B
:101A50000750F66E0900F550000A7F0BD8B412004B
:101A600025EC04F02AEF0DF0525332333220636F2D
:101A70006D6D616E64733A0A0D616E6E454E54452C
:101A8000522020202020646973706C61797320419A
:101A900044206368616E6E656C206E6E20636F75A6
:101AA0006E742E0A0D636E454E5445522020202040
:101AB0002020636C65617273206469676974616C6E
:101AC000206F7574707574206E2E0A0D42202020D0
:101AD000202020202020202020656E61626C65205F
:101AE0005755505F5049432070617373776F72642C
:101AF0002C2064656661756C74206E6F7420656E51
:101B000061626C65642C20736176656420696E2067
:101B1000454550524F4D2E0A0D6220202020202096
:101B200020202020202064697361626C6520575555
:101B30005F5049432070617373776F72642C206427
:101B4000656661756C74206E6F7420656E61626C81
:101B500065642C20736176656420696E204545506C
:101B6000524F4D2E0A0D44202020202020202020DE
:101B70002020206465627567206D6F64652C20638A
:101B80006F6E7469756E6F75736C79207072696EA3
:101B9000747320746865204144432076616C7565D8
:101BA000732E0A0D642020202020202020202020B9
:101BB0002073746F7073206465627567206D6F6445
:101BC000652E0A0D452020202020202020202020C6
:101BD00020656E61626C652073657269616C20704E
:101BE0006F72742073746172742075702064656CF8
:101BF00061792C2073657269616C20706F7274203A
:101C000077696C6C20626520656E61626C6564202A
:101C100061626F757420312E35206D696E75746543
:101C20007320616674657220706F776572207570BD
:101C30002C2064656661756C74206E6F2064656C21
:101C400061792C20736176656420696E204545506A
:101C5000524F4D2E0A0D65202020202020202020CC
:101C600020202064697361626C652073657269610C
:101C70006C20706F727420737461727420757020A0
:101C800064656C61792C2064656661756C74206E86
:101C90006F2064656C61792C2073617665642069BE
:101CA0006E204550524F4D2E0A0D476E6E6E454EBA
:101CB000544552202020207365747320636C6F6339
:101CC0006B2063616C6962726174696F6E2C207441
:101CD000696D6572312072656C6F6164206C6F771D
:101CE00020627974652C2064656661756C7420319E
:101CF00037352C20697320736176656420696E2006
:101D0000454550524F4D2E0A0D672020202020209F
:101D1000202020202020646973706C617973206317
:101D20006C6F636B2063616C6962726174696F6E62
:101D30002E0A0D486E6E454E54455220202020201C
:101D40007365747320686F75722E0A0D68202020E9
:101D500020202020202020202068656C702C2074FA
:101D60006869732068656C702E0A0D696E454E5463
:101D70004552202020202020726561647320646910
:101D8000676974616C20696E707574206E2E0A0D1F
:101D90004C2020202020202020202020206C6F6339
:101DA0006B7320746865205049432C20746865204B
:101DB0005049432077696C6C206E6F206C6F6E67A2
:101DC00065722070726F6365737320636F6D6D61F0
:101DD0006E64732C206F72207265706C7920746F42
:101DE00020636F6D6D616E64732C2057555F504991
:101DF000432077696C6C20656E61626C6520697444
:101E000020616761696E2E0A0D4D6E6E454E544518
:101E100052202020202073657473206D696E7574C4
:101E2000652E0A0D516E6E6E454E5445522020208F
:101E300020736574732050574D206F7574707574DE
:101E40002076616C7565206F6E2070696E20352E6E
:101E50000A0D712020202020202020202020206416
:101E60006973706C6179732070776D207365747419
:101E7000696E672E0A0D726E6E454E5445522020D3
:101E8000202020646973706C617973204144206361
:101E900068616E6E656C206E6E20636F6E76657223
:101EA00074656420746F2074656D706572617475FB
:101EB000726520696E2043656C6369757320666F77
:101EC00072206120636F6E6E6563746564204C4D93
:101ED0003133352073656E736F722E0A0D736E4544
:101EE0004E544552202020202020736574732064B6
:101EF00069676974616C206F7574707574206E2EDB
:101F00000A0D742020202020202020202020207056
:101F100072696E74732074696D652E0A0D766E6E2B
:101F2000454E5445522020202020646973706C6116
:101F30007973204144206368616E6E656C206E6E1B
:101F400020636F6E76657274656420746F20766F9F
:101F50006C746167652E0A0D57555F504943202008
:101F600020202020207468697320737472696E6762
:101F700020756E6C6F636B732074686520504943E5
:101F80002C206166746572207468617420737472A9
:101F9000696E6720746865205049432077696C6CCE
:101FA0002073656E642074686520494420616E6406
:101FB0002070726F6772616D2076657273696F6EE3
:101FC0002C20616E64207265706C7920746F2063C0
:101FD0006F6D6D616E64732E0A0D772020202020B6
:101FE00020202020202020646973706C6179732088
:101FF000686561746572206F6E2074696D65206913
:102000006E206D696E757465732C20686F757273C0
:102010002C20616E6420646179732E0A0D586E6EF7
:102020006E454E54455220202020736574732074F1
:10203000656D706572617475726520736574706F1B
:10204000696E742C20736176656420696E20454545
:1020500050524F4D2E207768656E205820697320AE
:102060003235352074686520746865726D6F7374DD
:102070006174206973206E6F74206F706572617473
:10208000696E672C20656C73650A0D202020202066
:1020900020202020202020202069662074686520D0
:1020A00074656D706572617475726520617420610C
:1020B0006E616C6F6720696E7075742041322028E4
:1020C00070696E20313729203C2074656D7065720F
:1020D00061747572655F736574706F696E742C20BE
:1020E0006469676974616C206F75747075742043DE
:1020F00030202870696E203136292069732073657D
:102100007420746F206C6F676963616C20273027BF
:102110002C0A0D20202020202020202020202020DC
:1021200020656C7365206469676974616C206F75E4
:1021300074707574204330202870696E2031362900
:102140002069732073657420746F206C6F676963F6
:10215000616C202731272C0A0D20202020202020F0
:10216000202020202020206E65676174697665201C
:10217000736574706F696E747320617265206E6F21
:102180007420737570706F727465642E0A0D7820F8
:102190002020202020202020202020646973706CC3
:1021A0006179732074656D706572617475726520F4
:1021B000736574706F696E742E0A0D59202020208B
:1021C000202020202020202070726F6772616D20F7
:1021D00074696D6572203120636F6D6D616E642C62
:1021E0002073657420686F75722C206D696E75742C
:1021F000652C20616E6420616E206173736F63696A
:1022000061746564206E65772074656D70657261B8
:10221000747572652C20736176656420696E204543
:102220004550524F4D2C207768656E20686F75724F
:10223000203E203233206F72206D696E75746520E8
:102240003E203539207468652074696D6572206997
:1022500073206E6F74206F7065726174696E672E83
:102260000A0D7920202020202020202020202070EE
:1022700072696E742074696D6572732E0A0D5A202E
:10228000202020202020202020202070726F6772C4
:10229000616D2074696D6572203220636F6D6D61B0
:1022A0006E642C2073657420686F75722C206D69C4
:1022B0006E7574652C20616E6420616E206173738D
:1022C0006F636961746564206E65772074656D70F5
:1022D000657261747572652C20736176656420691E
:1022E0006E20454550524F4D2C207768656E206812
:1022F0006F7572203E203233206F72206D696E75CB
:102300007465203E203539207468652074696D65D8
:1023100072206973206E6F74206F706572617469CA
:102320006E672E0A0D0A000050616E74656C746A47
:102330006520494F2D302E3720666F72205049435B
:0C2340002031384631344B32320D0A0097
:020000040030CA
:0E000000FF080714FF0041FF03C003E00340A8
:00000001FF
